 GetOwnedMonitorInfoWithEATest

 Timestamp is e4a4e964 (reproducible build file hash)

 Preferred load address is 0000000180000000

 Start         Length     Name                   Class
 0001:00000000 00001160H .text$mn                CODE
 0001:00001160 00000036H .text$mn$00             CODE
 0001:00001196 00000092H .text$x                 CODE
 0002:00000000 00000108H .idata$5                DATA
 0002:00000108 00000038H .00cfg                  DATA
 0002:00000140 00000008H .CRT$XCA                DATA
 0002:00000148 00000008H .CRT$XCZ                DATA
 0002:00000150 00000008H .CRT$XIA                DATA
 0002:00000158 00000008H .CRT$XIZ                DATA
 0002:00000160 00000008H .CRT$XPA                DATA
 0002:00000168 00000008H .CRT$XPZ                DATA
 0002:00000170 00000008H .CRT$XTA                DATA
 0002:00000178 00000008H .CRT$XTZ                DATA
 0002:00000180 00000000H .gehcont$y              DATA
 0002:00000180 00000000H .gfids$y                DATA
 0002:00000180 00000400H .rdata                  DATA
 0002:00000580 00000000H .rdata$CastGuardVftablesA DATA
 0002:00000580 00000000H .rdata$CastGuardVftablesC DATA
 0002:00000580 00000064H .rdata$voltmd           DATA
 0002:000005e4 000002acH .rdata$zzzdbg           DATA
 0002:00000890 00000008H .rtc$IAA                DATA
 0002:00000898 00000008H .rtc$IZZ                DATA
 0002:000008a0 00000008H .rtc$TAA                DATA
 0002:000008a8 00000008H .rtc$TZZ                DATA
 0002:000008b0 000001e0H .xdata                  DATA
 0002:00000a90 000000d0H .edata                  DATA
 0002:00000b60 00000050H .idata$2                DATA
 0002:00000bb0 00000018H .idata$3                DATA
 0002:00000bc8 00000108H .idata$4                DATA
 0002:00000cd0 000002e6H .idata$6                DATA
 0003:00000000 00000040H .data                   DATA
 0003:00000040 000005f8H .bss                    DATA
 0004:00000000 00000210H .pdata                  DATA

  Address         Publics by Value              Rva+Base               Lib:Object

 0000:00000000       __AbsoluteZero             0000000000000000     <absolute>
 0000:00000000       ___safe_se_handler_count   0000000000000000     <absolute>
 0000:00000000       ___safe_se_handler_table   0000000000000000     <absolute>
 0000:00000000       __arm64x_extra_rfe_table   0000000000000000     <absolute>
 0000:00000000       __arm64x_extra_rfe_table_size 0000000000000000     <absolute>
 0000:00000000       __arm64x_native_entrypoint 0000000000000000     <absolute>
 0000:00000000       __arm64x_redirection_metadata 0000000000000000     <absolute>
 0000:00000000       __arm64x_redirection_metadata_count 0000000000000000     <absolute>
 0000:00000000       __dynamic_value_reloc_table 0000000000000000     <absolute>
 0000:00000000       __enclave_config           0000000000000000     <absolute>
 0000:00000000       __guard_check_icall_a64n_fptr 0000000000000000     <absolute>
 0000:00000000       __guard_eh_cont_count      0000000000000000     <absolute>
 0000:00000000       __guard_eh_cont_table      0000000000000000     <absolute>
 0000:00000000       __guard_fids_count         0000000000000000     <absolute>
 0000:00000000       __guard_fids_table         0000000000000000     <absolute>
 0000:00000000       __guard_iat_count          0000000000000000     <absolute>
 0000:00000000       __guard_iat_table          0000000000000000     <absolute>
 0000:00000000       __guard_longjmp_count      0000000000000000     <absolute>
 0000:00000000       __guard_longjmp_table      0000000000000000     <absolute>
 0000:00000000       __hybrid_auxiliary_iat     0000000000000000     <absolute>
 0000:00000000       __hybrid_auxiliary_iat_copy 0000000000000000     <absolute>
 0000:00000000       __hybrid_code_map          0000000000000000     <absolute>
 0000:00000000       __hybrid_code_map_count    0000000000000000     <absolute>
 0000:00000000       __x64_code_ranges_to_entry_points 0000000000000000     <absolute>
 0000:00000000       __x64_code_ranges_to_entry_points_count 0000000000000000     <absolute>
 0000:00000100       __guard_flags              0000000000000100     <absolute>
 0000:00000000       __ImageBase                0000000180000000     <linker-defined>
 0001:0000010c       Agent_OnAttach             000000018000110c f   libGetOwnedMonitorInfoWithEATest.obj
 0001:0000010c       Agent_OnLoad               000000018000110c f   libGetOwnedMonitorInfoWithEATest.obj
 0001:00000114       JNI_OnLoad                 0000000180001114 f   libGetOwnedMonitorInfoWithEATest.obj
 0001:00000168       Java_GetOwnedMonitorInfoWithEATest_getOwnedMonitorInfo 0000000180001168 f   libGetOwnedMonitorInfoWithEATest.obj
 0001:000002fc       __local_stdio_printf_options 00000001800012fc f i libGetOwnedMonitorInfoWithEATest.obj
 0001:00000304       fprintf                    0000000180001304 f i libGetOwnedMonitorInfoWithEATest.obj
 0001:00000348       printf                     0000000180001348 f i libGetOwnedMonitorInfoWithEATest.obj
 0001:0000039c       __GSHandlerCheck           000000018000139c f   MSVCRT:gshandler.obj
 0001:000003bc       __GSHandlerCheckCommon     00000001800013bc f   MSVCRT:gshandler.obj
 0001:00000430       __security_check_cookie    0000000180001430 f   MSVCRT:amdsecgs.obj
 0001:00000770       _DllMainCRTStartup         0000000180001770 f   MSVCRT:dll_dllmain.obj
 0001:000007b0       __raise_securityfailure    00000001800017b0 f   MSVCRT:gs_report.obj
 0001:000007e4       __report_gsfailure         00000001800017e4 f   MSVCRT:gs_report.obj
 0001:0000092c       __security_init_cookie     000000018000192c f   MSVCRT:gs_support.obj
 0001:000009d8       DllMain                    00000001800019d8 f   MSVCRT:dll_dllmain_stub.obj
 0001:000009fc       ?__scrt_initialize_type_info@@YAXXZ 00000001800019fc f   MSVCRT:tncleanup.obj
 0001:00000a0c       ?__scrt_uninitialize_type_info@@YAXXZ 0000000180001a0c f   MSVCRT:tncleanup.obj
 0001:00000a18       __local_stdio_scanf_options 0000000180001a18 f i MSVCRT:default_local_stdio_options.obj
 0001:00000a20       __scrt_initialize_default_local_stdio_options 0000000180001a20 f   MSVCRT:default_local_stdio_options.obj
 0001:00000a3c       __scrt_acquire_startup_lock 0000000180001a3c f   MSVCRT:utility.obj
 0001:00000a78       __scrt_dllmain_after_initialize_c 0000000180001a78 f   MSVCRT:utility.obj
 0001:00000aac       __scrt_dllmain_before_initialize_c 0000000180001aac f   MSVCRT:utility.obj
 0001:00000ac4       __scrt_dllmain_crt_thread_attach 0000000180001ac4 f   MSVCRT:utility.obj
 0001:00000aec       __scrt_dllmain_crt_thread_detach 0000000180001aec f   MSVCRT:utility.obj
 0001:00000b04       __scrt_dllmain_exception_filter 0000000180001b04 f   MSVCRT:utility.obj
 0001:00000b64       __scrt_dllmain_uninitialize_c 0000000180001b64 f   MSVCRT:utility.obj
 0001:00000b94       __scrt_dllmain_uninitialize_critical 0000000180001b94 f   MSVCRT:utility.obj
 0001:00000ba8       __scrt_initialize_crt      0000000180001ba8 f   MSVCRT:utility.obj
 0001:00000bf4       __scrt_initialize_onexit_tables 0000000180001bf4 f   MSVCRT:utility.obj
 0001:00000c80       __scrt_is_nonwritable_in_current_image 0000000180001c80 f   MSVCRT:utility.obj
 0001:00000d18       __scrt_release_startup_lock 0000000180001d18 f   MSVCRT:utility.obj
 0001:00000d3c       __scrt_uninitialize_crt    0000000180001d3c f   MSVCRT:utility.obj
 0001:00000d68       __scrt_get_dyn_tls_init_callback 0000000180001d68 f   MSVCRT:dyn_tls_init.obj
 0001:00000d70       __crt_debugger_hook        0000000180001d70 f   MSVCRT:utility_desktop.obj
 0001:00000d78       __scrt_fastfail            0000000180001d78 f   MSVCRT:utility_desktop.obj
 0001:00000ec4       _RTC_Initialize            0000000180001ec4 f   MSVCRT:initsect.obj
 0001:00000f00       _RTC_Terminate             0000000180001f00 f   MSVCRT:initsect.obj
 0001:00000f3c       _guard_check_icall_nop     0000000180001f3c f i MSVCRT:guard_support.obj
 0001:00000f40       __isa_available_init       0000000180001f40 f   MSVCRT:cpu_disp.obj
 0001:000010ec       _get_startup_argv_mode     00000001800020ec f   MSVCRT:argv_mode.obj
 0001:000010f4       __scrt_is_ucrt_dll_in_use  00000001800020f4 f   MSVCRT:ucrt_detection.obj
 0001:00001100       memset                     0000000180002100 f   vcruntime:VCRUNTIME140.dll
 0001:00001106       __C_specific_handler       0000000180002106 f   vcruntime:VCRUNTIME140.dll
 0001:0000110c       __std_type_info_destroy_list 000000018000210c f   vcruntime:VCRUNTIME140.dll
 0001:00001112       _initterm                  0000000180002112 f   ucrt:api-ms-win-crt-runtime-l1-1-0.dll
 0001:00001118       _initterm_e                0000000180002118 f   ucrt:api-ms-win-crt-runtime-l1-1-0.dll
 0001:0000111e       _seh_filter_dll            000000018000211e f   ucrt:api-ms-win-crt-runtime-l1-1-0.dll
 0001:00001124       _configure_narrow_argv     0000000180002124 f   ucrt:api-ms-win-crt-runtime-l1-1-0.dll
 0001:0000112a       _initialize_narrow_environment 000000018000212a f   ucrt:api-ms-win-crt-runtime-l1-1-0.dll
 0001:00001130       _initialize_onexit_table   0000000180002130 f   ucrt:api-ms-win-crt-runtime-l1-1-0.dll
 0001:00001136       _execute_onexit_table      0000000180002136 f   ucrt:api-ms-win-crt-runtime-l1-1-0.dll
 0001:0000113c       _cexit                     000000018000213c f   ucrt:api-ms-win-crt-runtime-l1-1-0.dll
 0001:00001144       __acrt_initialize          0000000180002144 f   MSVCRT:ucrt_stubs.obj
 0001:00001144       __acrt_thread_attach       0000000180002144 f   MSVCRT:ucrt_stubs.obj
 0001:00001144       __acrt_thread_detach       0000000180002144 f   MSVCRT:ucrt_stubs.obj
 0001:00001144       __acrt_uninitialize        0000000180002144 f   MSVCRT:ucrt_stubs.obj
 0001:00001144       __acrt_uninitialize_critical 0000000180002144 f   MSVCRT:ucrt_stubs.obj
 0001:00001144       __scrt_stub_for_acrt_initialize 0000000180002144 f   MSVCRT:ucrt_stubs.obj
 0001:00001144       __scrt_stub_for_acrt_thread_attach 0000000180002144 f   MSVCRT:ucrt_stubs.obj
 0001:00001144       __scrt_stub_for_acrt_thread_detach 0000000180002144 f   MSVCRT:ucrt_stubs.obj
 0001:00001144       __scrt_stub_for_acrt_uninitialize 0000000180002144 f   MSVCRT:ucrt_stubs.obj
 0001:00001144       __scrt_stub_for_acrt_uninitialize_critical 0000000180002144 f   MSVCRT:ucrt_stubs.obj
 0001:00001144       __vcrt_initialize          0000000180002144 f   MSVCRT:ucrt_stubs.obj
 0001:00001144       __vcrt_thread_attach       0000000180002144 f   MSVCRT:ucrt_stubs.obj
 0001:00001144       __vcrt_thread_detach       0000000180002144 f   MSVCRT:ucrt_stubs.obj
 0001:00001144       __vcrt_uninitialize        0000000180002144 f   MSVCRT:ucrt_stubs.obj
 0001:00001144       __vcrt_uninitialize_critical 0000000180002144 f   MSVCRT:ucrt_stubs.obj
 0001:00001148       __scrt_stub_for_is_c_termination_complete 0000000180002148 f   MSVCRT:ucrt_stubs.obj
 0001:00001148       _is_c_termination_complete 0000000180002148 f   MSVCRT:ucrt_stubs.obj
 0001:0000114b       memcpy                     000000018000214b f   vcruntime:VCRUNTIME140.dll
 0001:00001170       _guard_dispatch_icall_nop  0000000180002170 f   MSVCRT:guard_dispatch.obj
 0001:00001190       _guard_xfg_dispatch_icall_nop 0000000180002190 f   MSVCRT:guard_xfg_dispatch.obj
 0002:00000000       __imp_RtlCaptureContext    0000000180003000     kernel32:KERNEL32.dll
 0002:00000008       __imp_RtlLookupFunctionEntry 0000000180003008     kernel32:KERNEL32.dll
 0002:00000010       __imp_RtlVirtualUnwind     0000000180003010     kernel32:KERNEL32.dll
 0002:00000018       __imp_UnhandledExceptionFilter 0000000180003018     kernel32:KERNEL32.dll
 0002:00000020       __imp_SetUnhandledExceptionFilter 0000000180003020     kernel32:KERNEL32.dll
 0002:00000028       __imp_GetCurrentProcess    0000000180003028     kernel32:KERNEL32.dll
 0002:00000030       __imp_TerminateProcess     0000000180003030     kernel32:KERNEL32.dll
 0002:00000038       __imp_IsProcessorFeaturePresent 0000000180003038     kernel32:KERNEL32.dll
 0002:00000040       __imp_QueryPerformanceCounter 0000000180003040     kernel32:KERNEL32.dll
 0002:00000048       __imp_GetCurrentProcessId  0000000180003048     kernel32:KERNEL32.dll
 0002:00000050       __imp_GetCurrentThreadId   0000000180003050     kernel32:KERNEL32.dll
 0002:00000058       __imp_GetSystemTimeAsFileTime 0000000180003058     kernel32:KERNEL32.dll
 0002:00000060       __imp_DisableThreadLibraryCalls 0000000180003060     kernel32:KERNEL32.dll
 0002:00000068       __imp_InitializeSListHead  0000000180003068     kernel32:KERNEL32.dll
 0002:00000070       __imp_IsDebuggerPresent    0000000180003070     kernel32:KERNEL32.dll
 0002:00000078       \177KERNEL32_NULL_THUNK_DATA 0000000180003078     kernel32:KERNEL32.dll
 0002:00000080       __imp_memset               0000000180003080     vcruntime:VCRUNTIME140.dll
 0002:00000088       __imp___C_specific_handler 0000000180003088     vcruntime:VCRUNTIME140.dll
 0002:00000090       __imp___std_type_info_destroy_list 0000000180003090     vcruntime:VCRUNTIME140.dll
 0002:00000098       __imp_memcpy               0000000180003098     vcruntime:VCRUNTIME140.dll
 0002:000000a0       \177VCRUNTIME140_NULL_THUNK_DATA 00000001800030a0     vcruntime:VCRUNTIME140.dll
 0002:000000a8       __imp__execute_onexit_table 00000001800030a8     ucrt:api-ms-win-crt-runtime-l1-1-0.dll
 0002:000000b0       __imp__initterm            00000001800030b0     ucrt:api-ms-win-crt-runtime-l1-1-0.dll
 0002:000000b8       __imp__initterm_e          00000001800030b8     ucrt:api-ms-win-crt-runtime-l1-1-0.dll
 0002:000000c0       __imp__seh_filter_dll      00000001800030c0     ucrt:api-ms-win-crt-runtime-l1-1-0.dll
 0002:000000c8       __imp__configure_narrow_argv 00000001800030c8     ucrt:api-ms-win-crt-runtime-l1-1-0.dll
 0002:000000d0       __imp__initialize_narrow_environment 00000001800030d0     ucrt:api-ms-win-crt-runtime-l1-1-0.dll
 0002:000000d8       __imp__initialize_onexit_table 00000001800030d8     ucrt:api-ms-win-crt-runtime-l1-1-0.dll
 0002:000000e0       __imp__cexit               00000001800030e0     ucrt:api-ms-win-crt-runtime-l1-1-0.dll
 0002:000000e8       \177api-ms-win-crt-runtime-l1-1-0_NULL_THUNK_DATA 00000001800030e8     ucrt:api-ms-win-crt-runtime-l1-1-0.dll
 0002:000000f0       __imp___stdio_common_vfprintf 00000001800030f0     ucrt:api-ms-win-crt-stdio-l1-1-0.dll
 0002:000000f8       __imp___acrt_iob_func      00000001800030f8     ucrt:api-ms-win-crt-stdio-l1-1-0.dll
 0002:00000100       \177api-ms-win-crt-stdio-l1-1-0_NULL_THUNK_DATA 0000000180003100     ucrt:api-ms-win-crt-stdio-l1-1-0.dll
 0002:00000108       __guard_check_icall_fptr   0000000180003108     MSVCRT:guard_support.obj
 0002:00000110       __guard_xfg_check_icall_fptr 0000000180003110     MSVCRT:guard_support.obj
 0002:00000118       __guard_dispatch_icall_fptr 0000000180003118     MSVCRT:guard_support.obj
 0002:00000120       __guard_xfg_dispatch_icall_fptr 0000000180003120     MSVCRT:guard_support.obj
 0002:00000128       __guard_xfg_table_dispatch_icall_fptr 0000000180003128     MSVCRT:guard_support.obj
 0002:00000130       __castguard_check_failure_os_handled_fptr 0000000180003130     MSVCRT:guard_support.obj
 0002:00000138       __guard_memcpy_fptr        0000000180003138     vcruntime:softmemtag.obj
 0002:00000140       __xc_a                     0000000180003140     MSVCRT:initializers.obj
 0002:00000148       __xc_z                     0000000180003148     MSVCRT:initializers.obj
 0002:00000150       __xi_a                     0000000180003150     MSVCRT:initializers.obj
 0002:00000158       __xi_z                     0000000180003158     MSVCRT:initializers.obj
 0002:00000160       __xp_a                     0000000180003160     MSVCRT:initializers.obj
 0002:00000168       __xp_z                     0000000180003168     MSVCRT:initializers.obj
 0002:00000170       __xt_a                     0000000180003170     MSVCRT:initializers.obj
 0002:00000178       __xt_z                     0000000180003178     MSVCRT:initializers.obj
 0002:00000180       ??_C@_0N@DGHLLIEK@?$CFs?3?5?$CFs?5?$CI?$CFd?$CJ?6@ 0000000180003180     libGetOwnedMonitorInfoWithEATest.obj
 0002:00000190       ??_C@_08KHBLFBMM@?$CFs?5?$CI?$CFd?$CJ?6@ 0000000180003190     libGetOwnedMonitorInfoWithEATest.obj
 0002:000001a0       ??_C@_0CA@OCHCPJ@Error?3?5GetEnv?5call?5failed?$CI?$CFd?$CJ?$CB?6@ 00000001800031a0     libGetOwnedMonitorInfoWithEATest.obj
 0002:000001c0       ??_C@_0BG@FLGBOFJG@Agent_OnLoad?5started?6@ 00000001800031c0     libGetOwnedMonitorInfoWithEATest.obj
 0002:000001d8       ??_C@_0DA@HOCMDKKL@Error?3?5wrong?5result?5of?5a?5valid?5@ 00000001800031d8     libGetOwnedMonitorInfoWithEATest.obj
 0002:00000208       ??_C@_0CN@NLBFDPME@Agent_OnLoad?3?5error?5in?5JVMTI?5Ad@ 0000000180003208     libGetOwnedMonitorInfoWithEATest.obj
 0002:00000238       ??_C@_0CN@FHMNLBKE@Agent_OnLoad?3?5error?5in?5JVMTI?5Ge@ 0000000180003238     libGetOwnedMonitorInfoWithEATest.obj
 0002:00000268       ??_C@_0DB@BAGELHMF@Warning?3?5GetOwnedMonitorInfo?5is@ 0000000180003268     libGetOwnedMonitorInfoWithEATest.obj
 0002:000002a0       ??_C@_0BH@NMEJPPEK@Agent_OnLoad?5finished?6@ 00000001800032a0     libGetOwnedMonitorInfoWithEATest.obj
 0002:000002b8       ??_C@_0DC@FFJMHPCJ@getOwnedMonitorsFor?3?5error?5in?5J@ 00000001800032b8     libGetOwnedMonitorInfoWithEATest.obj
 0002:000002f0       ??_C@_0DI@BOIGGMLJ@getOwnedMonitorsFor?3?5error?5in?5J@ 00000001800032f0     libGetOwnedMonitorInfoWithEATest.obj
 0002:00000328       ??_C@_0CM@HMKLKJJP@getOwnedMonitorsFor?3?5?$CFs?5owns?5?$CFd@ 0000000180003328     libGetOwnedMonitorInfoWithEATest.obj
 0002:00000358       _pDefaultRawDllMain        0000000180003358     MSVCRT:dll_dllmain.obj
 0002:00000358       _pRawDllMain               0000000180003358     MSVCRT:dll_dllmain.obj
 0002:00000370       __xmm@ffffffffffffffffffffffffffffffff 0000000180003370     MSVCRT:utility.obj
 0002:00000380       _load_config_used          0000000180003380     MSVCRT:loadcfg.obj
 0002:00000580       __volatile_metadata        0000000180003580     <linker-defined>
 0002:00000890       __rtc_iaa                  0000000180003890     MSVCRT:initsect.obj
 0002:00000898       __rtc_izz                  0000000180003898     MSVCRT:initsect.obj
 0002:000008a0       __rtc_taa                  00000001800038a0     MSVCRT:initsect.obj
 0002:000008a8       __rtc_tzz                  00000001800038a8     MSVCRT:initsect.obj
 0002:00000b60       __IMPORT_DESCRIPTOR_KERNEL32 0000000180003b60     kernel32:KERNEL32.dll
 0002:00000b74       __IMPORT_DESCRIPTOR_VCRUNTIME140 0000000180003b74     vcruntime:VCRUNTIME140.dll
 0002:00000b88       __IMPORT_DESCRIPTOR_api-ms-win-crt-stdio-l1-1-0 0000000180003b88     ucrt:api-ms-win-crt-stdio-l1-1-0.dll
 0002:00000b9c       __IMPORT_DESCRIPTOR_api-ms-win-crt-runtime-l1-1-0 0000000180003b9c     ucrt:api-ms-win-crt-runtime-l1-1-0.dll
 0002:00000bb0       __NULL_IMPORT_DESCRIPTOR   0000000180003bb0     kernel32:KERNEL32.dll
 0003:00000000       __security_cookie          0000000180004000     MSVCRT:gs_cookie.obj
 0003:00000008       __security_cookie_complement 0000000180004008     MSVCRT:gs_cookie.obj
 0003:00000010       __scrt_native_dllmain_reason 0000000180004010     MSVCRT:utility.obj
 0003:00000018       __isa_available            0000000180004018     MSVCRT:cpu_disp.obj
 0003:0000001c       __isa_enabled              000000018000401c     MSVCRT:cpu_disp.obj
 0003:00000020       __memset_fast_string_threshold 0000000180004020     MSVCRT:cpu_disp.obj
 0003:00000028       __memset_nt_threshold      0000000180004028     MSVCRT:cpu_disp.obj
 0003:00000030       __scrt_ucrt_dll_is_in_use  0000000180004030     MSVCRT:ucrt_stubs.obj
 0003:000005c0       ?__type_info_root_node@@3U__type_info_node@@A 00000001800045c0     MSVCRT:tncleanup.obj
 0003:000005d0       ?_OptionsStorage@?1??__local_stdio_scanf_options@@9@4_KA 00000001800045d0     MSVCRT:default_local_stdio_options.obj
 0003:000005d8       __scrt_current_native_startup_state 00000001800045d8     MSVCRT:utility.obj
 0003:000005e0       __scrt_native_startup_lock 00000001800045e0     MSVCRT:utility.obj
 0003:00000620       __scrt_debugger_hook_flag  0000000180004620     MSVCRT:utility_desktop.obj
 0003:00000624       __favor                    0000000180004624     MSVCRT:cpu_disp.obj
 0003:00000628       ?_OptionsStorage@?1??__local_stdio_printf_options@@9@9 0000000180004628     <common>
 0003:00000630       __dyn_tls_init_callback    0000000180004630     <common>

 entry point at        0001:00000770

 Static symbols

 0000:ffff9000       .debug$S                   0000000180000000     GetOwnedMonitorInfoWithEATest.exp
 0000:ffff9000       .debug$S                   0000000180000000     vcruntime:VCRUNTIME140.dll
 0000:ffff9000       .debug$S                   0000000180000000     vcruntime:VCRUNTIME140.dll
 0000:ffff9000       .debug$S                   0000000180000000     vcruntime:VCRUNTIME140.dll
 0000:ffff9000       .debug$S                   0000000180000000     vcruntime:VCRUNTIME140.dll
 0000:ffff9000       .debug$S                   0000000180000000     vcruntime:VCRUNTIME140.dll
 0000:ffff9000       .debug$S                   0000000180000000     vcruntime:VCRUNTIME140.dll
 0000:ffff9000       .debug$S                   0000000180000000     ucrt:api-ms-win-crt-runtime-l1-1-0.dll
 0000:ffff9000       .debug$S                   0000000180000000     ucrt:api-ms-win-crt-runtime-l1-1-0.dll
 0000:ffff9000       .debug$S                   0000000180000000     ucrt:api-ms-win-crt-runtime-l1-1-0.dll
 0000:ffff9000       .debug$S                   0000000180000000     ucrt:api-ms-win-crt-runtime-l1-1-0.dll
 0000:ffff9000       .debug$S                   0000000180000000     ucrt:api-ms-win-crt-runtime-l1-1-0.dll
 0000:ffff9000       .debug$S                   0000000180000000     ucrt:api-ms-win-crt-runtime-l1-1-0.dll
 0000:ffff9000       .debug$S                   0000000180000000     ucrt:api-ms-win-crt-runtime-l1-1-0.dll
 0000:ffff9000       .debug$S                   0000000180000000     ucrt:api-ms-win-crt-runtime-l1-1-0.dll
 0000:ffff9000       .debug$S                   0000000180000000     ucrt:api-ms-win-crt-runtime-l1-1-0.dll
 0000:ffff9000       .debug$S                   0000000180000000     ucrt:api-ms-win-crt-runtime-l1-1-0.dll
 0000:ffff9000       .debug$S                   0000000180000000     ucrt:api-ms-win-crt-runtime-l1-1-0.dll
 0000:ffff9000       .debug$S                   0000000180000000     ucrt:api-ms-win-crt-runtime-l1-1-0.dll
 0000:ffff9000       .debug$S                   0000000180000000     ucrt:api-ms-win-crt-stdio-l1-1-0.dll
 0000:ffff9000       .debug$S                   0000000180000000     ucrt:api-ms-win-crt-stdio-l1-1-0.dll
 0000:ffff9000       .debug$S                   0000000180000000     kernel32:KERNEL32.dll
 0000:ffff9000       .debug$S                   0000000180000000     kernel32:KERNEL32.dll
 0000:ffff9000       .debug$S                   0000000180000000     kernel32:KERNEL32.dll
 0000:ffff9000       .debug$S                   0000000180000000     kernel32:KERNEL32.dll
 0000:ffff9000       .debug$S                   0000000180000000     kernel32:KERNEL32.dll
 0000:ffff9000       .debug$S                   0000000180000000     kernel32:KERNEL32.dll
 0000:ffff9000       .debug$S                   0000000180000000     kernel32:KERNEL32.dll
 0000:ffff9000       .debug$S                   0000000180000000     kernel32:KERNEL32.dll
 0000:ffff9000       .debug$S                   0000000180000000     kernel32:KERNEL32.dll
 0000:ffff9000       .debug$S                   0000000180000000     kernel32:KERNEL32.dll
 0000:ffff9000       .debug$S                   0000000180000000     kernel32:KERNEL32.dll
 0000:ffff9000       .debug$S                   0000000180000000     kernel32:KERNEL32.dll
 0000:ffff9000       .debug$S                   0000000180000000     kernel32:KERNEL32.dll
 0000:ffff9000       .debug$S                   0000000180000000     kernel32:KERNEL32.dll
 0000:ffff9000       .debug$S                   0000000180000000     kernel32:KERNEL32.dll
 0000:ffff9000       .debug$S                   0000000180000000     kernel32:KERNEL32.dll
 0000:ffff9000       .debug$S                   0000000180000000     kernel32:KERNEL32.dll
 0001:00000000       Agent_Initialize           0000000180001000 f   libGetOwnedMonitorInfoWithEATest.obj
 0001:0000026c       ShowErrorMessage           000000018000126c f   libGetOwnedMonitorInfoWithEATest.obj
 0001:00000420       $$000000                   0000000180001420     MSVCRT:amdsecgs.obj
 0001:00000450       ?dllmain_crt_dispatch@@YAHQEAUHINSTANCE__@@KQEAX@Z 0000000180001450 f   MSVCRT:dll_dllmain.obj
 0001:000004a0       ?dllmain_crt_process_attach@@YAHQEAUHINSTANCE__@@QEAX@Z 00000001800014a0 f   MSVCRT:dll_dllmain.obj
 0001:000005b8       ?dllmain_crt_process_detach@@YAH_N@Z 00000001800015b8 f   MSVCRT:dll_dllmain.obj
 0001:0000063c       ?dllmain_dispatch@@YAHQEAUHINSTANCE__@@KQEAX@Z 000000018000163c f   MSVCRT:dll_dllmain.obj
 0001:000008b8       capture_previous_context   00000001800018b8 f   MSVCRT:gs_report.obj
 0001:00001160       $$000000                   0000000180002160     MSVCRT:guard_dispatch.obj
 0001:00001180       $$000000                   0000000180002180     MSVCRT:guard_xfg_dispatch.obj
 0001:00001196       ?fin$0@?0??dllmain_crt_process_attach@@YAHQEAUHINSTANCE__@@QEAX@Z@4HA 0000000180002196 f   MSVCRT:dll_dllmain.obj
 0001:000011ad       ?fin$0@?0??dllmain_crt_process_detach@@YAH_N@Z@4HA 00000001800021ad f   MSVCRT:dll_dllmain.obj
 0001:000011c6       ?fin$1@?0??dllmain_crt_process_detach@@YAH_N@Z@4HA 00000001800021c6 f   MSVCRT:dll_dllmain.obj
 0001:000011da       ?filt$0@?0??dllmain_dispatch@@YAHQEAUHINSTANCE__@@KQEAX@Z@4HA 00000001800021da f   MSVCRT:dll_dllmain.obj
 0001:00001210       __scrt_is_nonwritable_in_current_image$filt$0 0000000180002210 f   MSVCRT:utility.obj
 0002:00000360       GS_ExceptionPointers       0000000180003360     MSVCRT:gs_report.obj
 0002:000008b0       $unwind$fprintf            00000001800038b0     libGetOwnedMonitorInfoWithEATest.obj
 0002:000008bc       $unwind$printf             00000001800038bc     libGetOwnedMonitorInfoWithEATest.obj
 0002:000008c8       $unwind$JNI_OnLoad         00000001800038c8     libGetOwnedMonitorInfoWithEATest.obj
 0002:000008c8       $unwind$__raise_securityfailure 00000001800038c8     MSVCRT:gs_report.obj
 0002:000008c8       $unwind$__scrt_initialize_crt 00000001800038c8     MSVCRT:utility.obj
 0002:000008c8       $unwind$__scrt_initialize_onexit_tables 00000001800038c8     MSVCRT:utility.obj
 0002:000008c8       $unwind$__scrt_release_startup_lock 00000001800038c8     MSVCRT:utility.obj
 0002:000008c8       $unwind$__scrt_uninitialize_crt 00000001800038c8     MSVCRT:utility.obj
 0002:000008d0       $unwind$Agent_Initialize   00000001800038d0     libGetOwnedMonitorInfoWithEATest.obj
 0002:000008e0       $unwind$ShowErrorMessage   00000001800038e0     libGetOwnedMonitorInfoWithEATest.obj
 0002:000008f0       $unwind$Java_GetOwnedMonitorInfoWithEATest_getOwnedMonitorInfo 00000001800038f0     libGetOwnedMonitorInfoWithEATest.obj
 0002:00000904       $unwind$__GSHandlerCheckCommon 0000000180003904     MSVCRT:gshandler.obj
 0002:0000090c       $unwind$__scrt_initialize_default_local_stdio_options 000000018000390c     MSVCRT:default_local_stdio_options.obj
 0002:0000090c       $unwind$?dllmain_crt_dispatch@@YAHQEAUHINSTANCE__@@KQEAX@Z 000000018000390c     MSVCRT:dll_dllmain.obj
 0002:0000090c       $unwind$DllMain            000000018000390c     MSVCRT:dll_dllmain_stub.obj
 0002:0000090c       $unwind$__GSHandlerCheck   000000018000390c     MSVCRT:gshandler.obj
 0002:0000090c       $unwind$__scrt_acquire_startup_lock 000000018000390c     MSVCRT:utility.obj
 0002:0000090c       $unwind$__scrt_dllmain_after_initialize_c 000000018000390c     MSVCRT:utility.obj
 0002:0000090c       $unwind$__scrt_dllmain_before_initialize_c 000000018000390c     MSVCRT:utility.obj
 0002:0000090c       $unwind$__scrt_dllmain_crt_thread_attach 000000018000390c     MSVCRT:utility.obj
 0002:0000090c       $unwind$__scrt_dllmain_crt_thread_detach 000000018000390c     MSVCRT:utility.obj
 0002:0000090c       $unwind$__scrt_dllmain_uninitialize_c 000000018000390c     MSVCRT:utility.obj
 0002:0000090c       $unwind$__scrt_dllmain_uninitialize_critical 000000018000390c     MSVCRT:utility.obj
 0002:00000918       $xdatasym                  0000000180003918     MSVCRT:amdsecgs.obj
 0002:0000091c       $unwind$?dllmain_crt_process_attach@@YAHQEAUHINSTANCE__@@QEAX@Z 000000018000391c     MSVCRT:dll_dllmain.obj
 0002:00000958       $unwind$?fin$0@?0??dllmain_crt_process_attach@@YAHQEAUHINSTANCE__@@QEAX@Z@4HA 0000000180003958     MSVCRT:dll_dllmain.obj
 0002:00000958       $unwind$?fin$0@?0??dllmain_crt_process_detach@@YAH_N@Z@4HA 0000000180003958     MSVCRT:dll_dllmain.obj
 0002:00000958       $unwind$?fin$1@?0??dllmain_crt_process_detach@@YAH_N@Z@4HA 0000000180003958     MSVCRT:dll_dllmain.obj
 0002:00000960       $unwind$?dllmain_crt_process_detach@@YAH_N@Z 0000000180003960     MSVCRT:dll_dllmain.obj
 0002:000009b4       $unwind$?dllmain_dispatch@@YAHQEAUHINSTANCE__@@KQEAX@Z 00000001800039b4     MSVCRT:dll_dllmain.obj
 0002:000009dc       $unwind$?filt$0@?0??dllmain_dispatch@@YAHQEAUHINSTANCE__@@KQEAX@Z@4HA 00000001800039dc     MSVCRT:dll_dllmain.obj
 0002:000009e4       $unwind$_DllMainCRTStartup 00000001800039e4     MSVCRT:dll_dllmain.obj
 0002:000009f4       $unwind$__report_gsfailure 00000001800039f4     MSVCRT:gs_report.obj
 0002:000009fc       $unwind$capture_previous_context 00000001800039fc     MSVCRT:gs_report.obj
 0002:00000a08       $unwind$__security_init_cookie 0000000180003a08     MSVCRT:gs_support.obj
 0002:00000a14       $unwind$__scrt_is_nonwritable_in_current_image 0000000180003a14     MSVCRT:utility.obj
 0002:00000a34       $unwind$__scrt_is_nonwritable_in_current_image$filt$0 0000000180003a34     MSVCRT:utility.obj
 0002:00000a3c       $unwind$__scrt_dllmain_exception_filter 0000000180003a3c     MSVCRT:utility.obj
 0002:00000a50       $unwind$__scrt_fastfail    0000000180003a50     MSVCRT:utility_desktop.obj
 0002:00000a60       $unwind$_RTC_Initialize    0000000180003a60     MSVCRT:initsect.obj
 0002:00000a60       $unwind$_RTC_Terminate     0000000180003a60     MSVCRT:initsect.obj
 0002:00000a6c       $unwind$__isa_available_init 0000000180003a6c     MSVCRT:cpu_disp.obj
 0002:00000a80       $xdatasym                  0000000180003a80     MSVCRT:guard_dispatch.obj
 0002:00000a88       $xdatasym                  0000000180003a88     MSVCRT:guard_xfg_dispatch.obj
 0002:00000a90       .edata                     0000000180003a90     GetOwnedMonitorInfoWithEATest.exp
 0002:00000ab8       rgpv                       0000000180003ab8     GetOwnedMonitorInfoWithEATest.exp
 0002:00000ac8       rgszName                   0000000180003ac8     GetOwnedMonitorInfoWithEATest.exp
 0002:00000ad8       rgwOrd                     0000000180003ad8     GetOwnedMonitorInfoWithEATest.exp
 0002:00000ae0       szName                     0000000180003ae0     GetOwnedMonitorInfoWithEATest.exp
 0002:00000b02       $N00001                    0000000180003b02     GetOwnedMonitorInfoWithEATest.exp
 0002:00000b11       $N00002                    0000000180003b11     GetOwnedMonitorInfoWithEATest.exp
 0002:00000b1e       $N00003                    0000000180003b1e     GetOwnedMonitorInfoWithEATest.exp
 0002:00000b29       $N00004                    0000000180003b29     GetOwnedMonitorInfoWithEATest.exp
 0002:00000e36       .idata$6                   0000000180003e36     kernel32:KERNEL32.dll
 0002:00000e86       .idata$6                   0000000180003e86     vcruntime:VCRUNTIME140.dll
 0002:00000f6a       .idata$6                   0000000180003f6a     ucrt:api-ms-win-crt-stdio-l1-1-0.dll
 0002:00000f8a       .idata$6                   0000000180003f8a     ucrt:api-ms-win-crt-runtime-l1-1-0.dll
 0003:00000040       jvmti                      0000000180004040     libGetOwnedMonitorInfoWithEATest.obj
 0003:00000048       ?__proc_attached@@3HA      0000000180004048     MSVCRT:dll_dllmain.obj
 0003:00000050       GS_ExceptionRecord         0000000180004050     MSVCRT:gs_report.obj
 0003:000000f0       GS_ContextRecord           00000001800040f0     MSVCRT:gs_report.obj
 0003:000005e8       ?is_initialized_as_dll@@3_NA 00000001800045e8     MSVCRT:utility.obj
 0003:000005e9       ?module_local_atexit_table_initialized@@3_NA 00000001800045e9     MSVCRT:utility.obj
 0003:000005f0       ?module_local_atexit_table@@3U_onexit_table_t@@A 00000001800045f0     MSVCRT:utility.obj
 0003:00000608       ?module_local_at_quick_exit_table@@3U_onexit_table_t@@A 0000000180004608     MSVCRT:utility.obj
